:020000040000FA
:06000000D9EF0EF0120022
:06080000D9EF0EF012001A
:06082A0001001A1E00008F
:08083000000200002E00000090
:0808380058EC09F0FB0EDBCFC8
:10084000F3FFDB06F35000090AE0A6EC09F0FA0E0C
:1008500011EC0AF0F3E1151CF1E1010E01D0000EDC
:1008600087EF09F058EC09F03B0EE12402E3E16860
:10087000E652E16E010EDB6A020EDB6AF90EDBCF97
:10088000F6FFFA0EDBCFF7FFFB0EDBCFF8FF080019
:10089000F550DF6EDF5002E1ABEF08F0250EDF5CB4
:1008A00002E09EEF08F0030EDB6A040EDB6A050E21
:1008B000DB6A060EDB6A070EDB6AC0EC08F02D0E61
:1008C000DF5C0CE02B0EDF5C09E0200EDF5C06E055
:1008D000230EDF5C03E0300EDF5C1AE1DF50300AEC
:1008E00014E0130A0FE0030A0AE00B0A05E0060A07
:1008F000E4E1030EDB80E1D7030EDB82DED7030EDB
:10090000DB84DBD7030EDB86D8D7030EDB88D5D795
:100910002A0EDF5C1BE1BCEC08F00AEC09F010E0E9
:10092000030EDB8008680968130EDBCF0DF0140E90
:10093000DBCF0EF056EC0EF0040E06C0DBFF03D04A
:10094000130EF3EC08F0C0EC08F00BD0090EDB6AD4
:1009500061EC09F003E0D5EC09F0FAD7090EF3ECED
:1009600008F0030EDBB0DB982E0EDF5C1BE1C0EC61
:1009700008F02A0EDF5C0BE1BCEC08F00AEC09F091
:1009800003E1130E45EC09F0C0EC08F00BD0090EA2
:10099000DB6A61EC09F003E0D5EC09F0FAD7090E47
:1009A00045EC09F0680EDF5C07E1C0EC08F0680E6A
:1009B000DF5C1DE1030E18D0740EDF5C17E07A0EC9
:1009C000DF5C14E0480EDF5C06E0540EDF5C03E001
:1009D0005A0EDF5C02E1020E07D06C0EDF5C03E012
:1009E0006A0EDF5C04E1010E98EC09F0C9DBDF5010
:1009F0006E0A01E17FD31E0A01E192D1200A01E1D2
:100A00008FD13F0A01E149D11A0A01E146D10D0A0D
:100A100001E143D1200A01E140D13A0A01E13DD18F
:100A2000200A01E13AD1260A01E135D10D0A01E19E
:100A300032D11A0A01E1D9D0200A4AE0300A1FE077
:100A4000460A0EE0250A01E083D3D950F90FE96E7A
:100A5000FF0EDA20EA6E010EEE5E000EEE5AEE5A3E
:100A6000A6EC09F0250EE66E95DB03E1151C01E10D
:100A700069D3A2EC09F001E26BD3DB2A69D3080E3B
:100A8000DB6A040EDB50010806E2040EDB046AECAC
:100A900009F0DB508BDB080EDB5009E0030EDB5066
:100AA000010B05E172DB01E04DD3080EDB6A64DB6C
:100AB000EFCFDFFF1AEC0AF003E1151C01E142D38E
:100AC000A2EC09F001E3DB2A60DB01E141D33AD378
:100AD000070EDB5002080FE1E6EC09F0030EADEC67
:100AE00009F00E0EEECFDBFF0F0EEECFDBFF100E88
:100AF000EECFDBFF20D0F70EDBCF17F0F80EDBCF09
:100B000018F0020E175E000E185AF70E17C0DBFF22
:100B1000F80E18C0DBFF17C0E9FF18C0EAFF9DEC14
:100B200009F0166A0E0E14C0DBFF0F0E15C0DBFFB6
:100B3000100E16C0DBFF0E0EDBCFE6FF0F0EDBCF75
:100B4000E6FF100EDBCFE6FF31EC0EF0E552E5528A
:100B5000E552130E07C0DBFF140E08C0DBFF060EC4
:100B6000DB5005E0130EE1EC09F001E26ADB05EC75
:100B70000AF002E2130E37DBC8EC09F006E0040EBF
:100B8000E1EC09F002E2050E2EDB030EDBB005D02E
:100B9000FCDA01E0D7D2080EDB6A090EDB6A0E0E22
:100BA000DBCFF6FF0F0EDBCFF7FF100EDBCFF8FF2A
:100BB0000800F550DF6EDF5014E00BEC0AF011E294
:100BC0001AEC0AF003E1151C01E1BCD2BBDB01E326
:100BD000DB2A090EDB2AD9500E0FE96E000ECBDBA3
:100BE000E7D7D3DA01E1B4D2ADD2C6DA110EEECF37
:100BF000DBFF120EEDCFDBFF110EDBCFE6FF120E97
:100C0000DBCFE6FF23EC0EF0E552E552130EF3CFF7
:100C1000DBFF140EF4CFDBFF060EDB5004E0130EF7
:100C2000D0DB01E20EDB05EC0AF002E2130EDBDAA8
:100C3000AFDB05E0040EC5DB02E2050ED4DA030EDD
:100C4000DBB005D0A2DA01E07DD2080EDB6A090E26
:100C5000DB6A110EDBCFE9FF120EDBCFEAFFEFCF2D
:100C6000DFFFDF5014E0D7DB12E2E4DB03E1151C09
:100C700001E168D267DB01E3DB2A090EDB2A110EF2
:100C8000DB2ADBCFE9FF120EE8E3DB2AE6D77DDAC9
:100C900001E15ED257D2030EDB8E070EDB0410E1BA
:100CA00095DB040E5ADB0A0EEECFDBFF0B0EEECF08
:100CB000DBFF0C0EEECFDBFF0D0EEECFDBFF6CD0BB
:100CC000070EDB5003082CE1030EDBAE0DD0B2DAC9
:100CD000020E76DAEFCF14F0156A166A176A14AEB0
:100CE00039D01568166835D0F70EDBCF15F0F80E41
:100CF000DBCF16F0020E155E000E165AF70E15C069
:100D0000DBFFF80E16C0DBFF15C0E9FF16C0EAFFD7
:100D1000EFCF14F00A0E14C0DBFF0B0EDB6A38D0E5
:100D2000070EDB50020809E1030EDBAE04D059DBED
:100D300016AE10D00ED055DB0DD0030EDBAE12D0A8
:100D400079DA020E3DDAF9DA166A176A15AE02D0C0
:100D500016681768E2DA0C0E16C0DBFF0D0E17C01E
:100D6000DBFF1AD0F70EDBCF16F0F80EDBCF17F053
:100D7000020E165E000E175AF70E16C0DBFFF80EB5
:100D800017C0DBFF16C0E9FF17C0EAFFD6DAC5DAE5
:100D90000C0EDB6A0D0EDB6A060EDB5005E1010E60
:100DA000F36E050EF3CFDBFF150EDB6A160EDB6A62
:100DB000D950370F146E000EDA20156E390E14C09C
:100DC000DBFF3A0E15C0DBFF380EDB6A080EDB6A6C
:100DD0000A0EAEDADF50780A12E0200A10E0280A84
:100DE0000CE0200A0AE03F0A06E00D0A02E0200AB1
:100DF00008E1020E05D0080E03D0080EDF26100E03
:100E000097DA030EDBBE02D0DB92DB94DB50800B63
:100E100024E08ADAD890030EEB50000A08E6000EB0
:100E2000EE5C000EEE58000EEE58000EEE5815E285
:100E300013DA0B680C680D680E68EBEC0DF00A0E07
:100E400002C0DBFF0B0E03C0DBFF0C0E04C0DBFF98
:100E50000D0E05C0DBFF2D0E08D0030EDBA202D065
:100E60002B0E03D0DBA408D0200EF36E170EF3CFA9
:100E7000DBFF150EDB2A02D0170EDB6A050EDB50F6
:100E800003E1B7D901E189D0000E146E1E0E156E74
:100E9000000E166E070EDBCF17F0186A196A1A6A71
:100EA00017C00BF018C00CF019C00DF01AC00EF0EE
:100EB000D3D983EC0EF014500224F36E15500320A6
:100EC000F46E16500420F86EF4CFF7FFF3CFF6FF60
:100ED0000800090EF5CFDBFF580EDF5C0FE1610E55
:100EE000F36E090E7BD90AE3200E146E090EDBCFD8
:100EF000E7FF1450E75E090EE7CFDBFF070EDBCFFD
:100F000014F0156A166A176A0FDA14C00BF015C0D0
:100F10000CF016C00DF017C00EF0EECF06F0EECFBD
:100F200007F0EECF08F0EFCF09F083EC0EF009C028
:100F3000EDFF08C0EDFF07C0EDFF06C0EFFF390E63
:100F4000DBCFE9FFDB063A0EDBCFEAFF01E2DB068F
:100F5000090EDBCFEFFF150EDB2A4BD995E1030E0F
:100F6000DBA61DD06F0EDF5C06E1C1D918E3150EBC
:100F7000DB285BDA14D0780EDF5C09E0580EDF5C0A
:100F800006E0620EDF5C03E0420EDF5C08E1020E69
:100F9000F36E160EF3CFDBFF02D0150EDB6A030EE5
:100FA000DB50100B0EE0040EDBCF14F0050EDB500F
:100FB000D880145406E2060EDB5003E1040EDB5029
:100FC00034DA95D90AE2050EDBCFE7FF150EDB50C8
:100FD000E75E050EE7CFDBFF02D0050EDB6A040EED
:100FE000DBCF14F0160E45D9D880145414E2160E37
:100FF000DBCFE6FF150EDBCFE6FF040EDBCFE6FF0F
:10100000050EDB50E552E75CE552D880E754E55227
:10101000D880E7545FD9030EDB50010B0BE1080EBB
:10102000DB5008E0B2D801E08DD0080EDB50BED80E
:10103000080EDB6A170EDB5007E088D9170EF1D9CE
:1010400003E1151C01E17ED0160EDB5016E07ED9BF
:10105000300EE66E9FD802E1151C74E077D9DFCF21
:10106000E6FFA9EC0DF0E552E552E552F4CF15F09C
:101070000001F31C02E1151C65E0050EDBCF14F046
:10108000160EDB50D880145409E2050EDBCFE7FFC3
:10109000160EDB50E75E050EE7CFDBFF300EE66E87
:1010A000050ECBD94FE1390EDB2ADBCFE9FF3A0E33
:1010B00001E3DB2ADBCFEAFF090EEFCFDBFFDB50DA
:1010C0000EE044D9090EADD902E1151C3BE0390E02
:1010D000DB2ADBCFE9FF3A0EEDE3DB2AEBD755D86D
:1010E00031E1160EDBCFE6FF080EC3D8E552E72448
:1010F0005DD82ED0070EDB50030A1CE0010A14E075
:10110000030A07E07BD9DBCFEEFF020EDBCFEDFF5A
:101110001FD0F5D8196A17AE02D0186819682CD8F4
:10112000BCD819C0EEFF14D0EAD817BE186824D86E
:10113000B4D80ED063D9DBCFEFFF0AD07BD905E15D
:10114000151C03E1F368F46810D0FCD801E3DB2A36
:1011500079D947EF04F0010EDBCF14F0020EDBCF9C
:1011600015F014C0F3FF15C0F4FF3B0EE15C02E282
:10117000E16AE552E16ECBD029D9020EADEF09F05C
:1011800061D90800F550DF6E1200200EE66E080EE1
:101190001DEF0AF0A9EC0DF0E552E552E552F3CF50
:1011A00014F0F4CF15F00001F31C1200146E156A50
:1011B000D950010F4DD91450EE261550ED221200D2
:1011C000185E000E195AF70E18C0DBFFF80E19C092
:1011D000DBFF18C0E9FF19C0EAFF1200DBCFF4FF04
:1011E000F350F45C1200DB50E76E040EE7CFDBFF38
:1011F00012000A0EDBCF14F00B0EDBCF15F00C0E35
:10120000DBCF16F00D0EDBCF17F0145015101610B3
:1012100017101200130EEECFDBFF140EEDCFDBFF25
:10122000130EDBCF14F0140EDBCF15F00001800E8F
:1012300015141200F70EDBCF18F0F80EDBCF19F003
:101240001200050EDB50E66ED950130F01D9E5529E
:10125000E750EE6EED6A12000A0EDBCF06F00B0EC1
:10126000DBCF07F00C0EDBCF08F00D0EDBCF09F063
:101270001200DBCFE6FF150EDBCFE6FF050EDB50DD
:10128000E552E724E552E7241200DB50CED8010EE8
:10129000F36E060EF3CFDBFF1200EE50EFCFEAFF46
:1012A000E96E16C0EEFF17C0EEFF18C0EEFF120089
:1012B000D9CFE6FFDACFE6FFE1CFD9FFE2CFDAFF01
:1012C0001200DFCFE6FFE66AA7EC0EF0E552E5522A
:1012D000F3501200E76E080EE7CFDBFF1200EECFEF
:1012E00014F0EECF15F0EFCF16F0176A1200050ECE
:1012F000DBCF14F0150EDB50D88014541200010E11
:10130000DBCF16F0020EDBCF17F0186A1200E552A1
:10131000E5CFDAFFE7CFD9FF12000A0E14C0DBFFDA
:101320000B0E15C0DBFF1200D9500A0F28EF0AF090
:10133000F36E070EF3CFDBFF1200EECF14F0EFCF0A
:1013400015F01200010EDB2A020E1200FC0EDBCF9C
:10135000E6FFFD0EDBCFE6FF1200145E000E155A0D
:10136000F70E14C0DBFFF80E15C0DBFF14C0E9FF59
:1013700015C0EAFF1200DA20EA6EEF2AEECFF6FF80
:10138000000EEF22EECFF7FFEF22EECFF8FF1200B4
:10139000040EDBCFE6FF130EDB50E552E75C9ADF6D
:1013A000DB5004DF060EDB501200090EDB500A0D85
:1013B000F350DF24D00FE76E090EE7CFDBFFC0EF5D
:1013C00008F0DB50F36E050EEEEF08F0F70EDBCF02
:1013D00014F0F80EDBCF15F01200DFCFE6FFCAEFF6
:1013E00008F028DF030EECDE6FEF09F01CEC04F0D0
:1013F000E552E552E552E55200091200BDDEEE501D
:10140000EFCFEAFFE96E010E1200130EDB50F36E10
:10141000040EEEEF08F0040EDB50F36E090EEEEF53
:1014200008F0DBCFE6FFCAEF08F0E76E050EE7CF66
:10143000DBFF12008BDFEDEF09F0DBCFE6FF86DF8D
:10144000F6EF09F0D950F90FE96EFF0EBBEF09F086
:0A145000E96E000EDA20EA6E1200C9
:06145A00D9CFE6FFE1CF4F
:10146000D9FF040EE126DE6ADE6ADE6ADD6ADD523D
:10147000DD52FD0EDBCF14F0FE0EDBCF15F0166A49
:10148000176A15AE02D016681768D9CFE9FFDACF10
:10149000EAFF030EEB501718E8AE02D0173408D05D
:1014A0001450EE5C1550EE581650EE581750EE588A
:1014B0000FE20C0EE66EB9EC0EF0E552D9CFE9FF63
:1014C000DACFEAFFEE2A000EEE22EE22EE22D1D78C
:1014D000040EE15C02E2E16AE552E16EE552E7CF1B
:1014E000D9FF12000F0EC16E070EB46E936A816AA7
:1014F000300E926E80900F0E946EF19E1200D9CF36
:10150000E6FFE1CFD9FF020EE1268250020B01E097
:10151000010E080DF3CF16F08250010B040DF3CF2E
:1015200015F08050200B01E0010EE824146E80506D
:10153000100B01E0010E142415241624DE6EDD6A62
:10154000DECF14F0DDCF15F014C0F3FF15C0F4FFAB
:10155000020EE15C03E200D0E16AE552E16EE55281
:10156000E7CFD9FF12008092320EE66EF5EC0EF056
:10157000E5528084320EE66EF5EC0EF0E552809472
:10158000320EE66EF5EC0EF0E55212008082010E8E
:10159000E66EE66A62DFE552E5528084010EE66E91
:1015A000E66A5BDFE552E5528094010EE66EE66A7C
:1015B00054DFE552E5521200380E816ED4DF320E50
:1015C000E66EE66A4ADFE552E552010E816ECBDF38
:1015D000320EE66EE66A41DFE552E5520D0E816E8F
:1015E000C2DF320EE66EE66A38DFE552E552060EDD
:1015F000816EB9DF320EE66EE66A2FDFE552E55204
:101600001200010E816EAFDF0A0EE66EE66A25DF7C
:10161000E552E5521200D9CFE6FFE1CFD9FF020E25
:10162000816EA1DF0A0EE66EE66A17DFE552E5522B
:10163000FD0EDBCFE6FFFE0EDB50280DF350E5522A
:10164000E724E76EFE0EE7CFDBFFFD0EDB6AFE0E42
:10165000DB50F36EFD0EDBCFF4FFF350F45C0BE2D6
:10166000140E816E80DF320EE66EF5EC0EF0E55260
:10167000FD0EDB2AECD7E552E7CFD9FF1200D9CF18
:10168000E6FFE1CFD9FFFE0EDB50816E7FDF010E5A
:10169000E66EE66AE2DEE552E552E552E7CFD9FFB3
:1016A0001200D9CFE6FFE1CFD9FFFD0EDBCFE9FF76
:1016B000FE0EDBCFEAFFEF500EE0FD0EDBCFE9FFC1
:1016C000DB2AFE0EDBCFEAFF01E3DB2AEF50E66EFA
:1016D000D6DFE552EAD7E552E7CFD9FF1200000185
:1016E000646B300E926EF00E936EEF0E606F60C002
:1016F00081FF040E616F6151000821E26051FE0B11
:10170000E842606F60C081FF050EE66EE66AA5DE06
:10171000E552E5528150100B09E08150200B06E0A4
:101720008150400B03E08150800B01E10AD8000199
:10173000640502E1655104D06105616FDCD7CFD744
:101740001200F00E936E81CF63F000016315626F9B
:101750000F0E6015606F60516211606F81CF63F092
:10176000F00E6315626FF00E625D01E0F7D7936AC9
:1017700006D866C065F00001010E646F120000011A
:10178000676B100E675D14E26751EA6A000FE96E3D
:10179000020EEA22EF50605D08E16751EA6A100F1D
:1017A000E96E020EEA22EFCF66F06729676FE9D78C
:1017B00066C081FF640EE66EE66A4FDEE552E552D2
:1017C00012000001686B070E685D1DE288DF0001F2
:1017D000696F6851EA6A6A0FE96E000EEA2269C011
:1017E000EFFF6851EA6A6A0FE96E000EEA22EF50D5
:1017F000460802E108D004D069C0E6FF40DFE552A8
:101800000001682BE0D76851EA6A6A0FE96E000EA2
:10181000EA22EF6A12000001686B070E685D16E2AB
:101820006851EA6A6A0FE96E000EEA22EF50E66E2E
:1018300026DFE55200016829EA6A6A0FE96E000EA8
:10184000EA22EF5001E102D0682BE7D71200D9CF8E
:10185000E6FFE1CFD9FFE652F250800B01E0010E26
:10186000DF6EF29EA69EA69CA684FE0EDB50A96E9D
:10187000FD0EDB50A86E550EA76EAA0EA76EA682AF
:10188000A6B2FED7A694DF50E8B0F28EE8A0F29E92
:10189000E552E552E7CFD9FF1200D9CFE6FFE1CFFD
:1018A000D9FFA69CA69EFE0EDB50A96EA680A8506E
:1018B00000D0E552E7CFD9FF12000001736B746BC3
:1018C00011DE0001732B000E7423E80E731902E180
:1018D000030E741902E1736B746B73C0E6FF74C07E
:1018E000E6FF110E146E1E0E156E166A14C0E6FF8A
:1018F00015C0E6FF16C0E6FF2A0EE66E020EE66E83
:1019000004EC0DF0176E070EE15E1750640E000137
:1019100074AF02D0D89003D0735D000E745903E207
:101920000201300E2A6F0A0E000174AF02D0D89067
:1019300003D0735D000E745904E20201300E2A6F69
:101940002B6F0001756B766B140E76AF02D0D890BA
:1019500003D0755D000E76591DE280828092776B10
:10196000786B030E78AF02D0D89003D0775D000E6D
:1019700078590CE22A0EE66E020EE66E0DD8E5529C
:10198000E5520001772B000E7823EBD7752B000E64
:101990007623DAD796D71200D9CFE6FFE1CFD9FF69
:1019A000020EE12680848094FD0EDB500001772535
:1019B0000F01E96EFE0EDB50000178210F01EA6E87
:1019C000EF50D00F146E156A14BE156814C0DEFFF8
:1019D00015C0DDFFDECFE9FFDDCFEAFF200EE926EF
:1019E000020EEA22EF50816E050EE66EE66A35DDE4
:1019F000E552E552020EE15C02E2E16AE552E16E77
:081A0000E552E7CFD9FF120007
:081A0800D9CFE6FFDACFE6FFBB
:101A1000E1CFD9FFE2CFDAFFE652E652E652E652D4
:101A2000D950F90F146EFF0EDA20156E020E14C095
:101A3000DBFF030E15C0DBFF020EDBCFE6FF030E5C
:101A4000DBCFE6FFF90EDBCFE6FFFA0EDBCFE6FFDA
:101A5000FB0EDBCFE6FFD950FC0FE66EFF0EDA205F
:101A6000E66E32EC04F0146E070EE15C02E2E16A0D
:101A7000E552E16E1450F3CFDEFFF4CFDDFFFC0E34
:101A8000DBCFE9FFFD0EDBCFEAFFEF6ADECF14F01C
:101A9000DDCF15F014C0F3FF15C0F4FF040EE15CB8
:101AA00002E2E16AE552E16EE552E5CFDAFFE7CF07
:041AB000D9FF120048
:0C1AB4002A0EF66E080EF76E000EF86E9B
:101AC00002010900F550336F0900F550346F03E14E
:101AD000336701D03DD00900F5502E6F0900F55055
:101AE0002F6F0900F550306F09000900F550E96EBD
:101AF0000900F550EA6E090009000900F550316F40
:101B00000900F550326F09000900F6CF35F2F7CF22
:101B100036F2F8CF37F22EC2F6FF2FC2F7FF30C2EF
:101B2000F8FF0201315302E1325307E00900F5509A
:101B3000EE6E3107F8E23207F9D735C2F6FF36C24A
:101B4000F7FF37C2F8FF02013307000E345BBFD73F
:021B5000120081
:0E1B5200D9CFE6FFDACFE6FFE1CFD9FFE2CF31
:101B6000DAFFFB0EDBCF14F0FC0EDBCF15F000012B
:101B7000800E15141AE1FB0EDBCFE9FFFC0EDBCF64
:101B8000EAFFEECFF3FFEDCFF4FFEE2A000EEF22D7
:101B9000F3CFE9FFF4CFEAFFFD0EDBCFEFFFEF500D
:101BA000156AF36E15C0F4FF10D0FB0EDB50FE0873
:101BB00006E1FD0EDBCFE6FFE7EC0EF005D0FD0EF3
:101BC000DBCFE6FF0BEC0FF0E552E552E5CFDAFF95
:061BD000E7CFD9FF12006F
:0A1BD60006500B02F3CF02F0F4CF2B
:101BE00003F00C02F3500326000EF420046E06509E
:101BF0000D02F3500426000EF420056E06500E026E
:101C0000F350052607500B02F3500326F45004222C
:101C1000000E052207500C02F3500426F450052252
:101C200007500D02F350052608500B02F35004260E
:101C3000F450052208500C02F350052609500B02FF
:061C4000F350052612001E
:0A1C4600FE0EE3CFE9FFFF0EE3CF2F
:101C5000EAFFF36AF46AEE5203E0F34AF42AFBD790
:101C60001200FF0EE3CFF8FFE552FF0EE3CFF7FFC0
:101C7000E552FF0EE3CFF6FFE552E66AE66AE66A52
:101C80000900F55209E0FD0EE32A05E1FE0EE32A04
:101C900002E1FF0EE32AF4D7FD0EE3CF07F0FE0EBC
:0C1CA000E3CF08F0FF0EE3CF09F01200C4
:041CAC0009C013F068
:101CB00008C012F008500D02F4CF07F0F3CF06F081
:101CC00009500E02F4CF09F0F3CF08F00D02F350E3
:101CD0000726F4500822E86A092212500E02F35037
:101CE0000726F4500822E86A09220EAE7CEF0EF0B7
:101CF0001250085E1350095A13AE000C0D50085EC6
:061D00000E50095A000C10
:0A1D0600056A046A036A026A200EEF
:101D1000E76ED8900636073608360936023603369F
:101D2000043605360B50025C0C5003580D50045815
:101D30000E50055809E30B50025E0C50035A0D502B
:0E1D4000045A0E50055A062AE72EE4D7120068
:021D4E00F36A36
:101D5000F46AFF0EE124E96EFF0EE220EA6EED6602
:101D600007D02F0EEF6404D03A0EEF6001D0F32AB3
:021D700012005F
:0E1D7200FF0EE3501B6E480E01D04C0EE76EC4
:101D8000E72EFED7E76AE72EFED71B2EF7D7000017
:021D900012003F
:0E1D9200000EF36E00EE00F0080E01D81200F5
:101DA000EA6002D0EE6AFCD7F350E9601200EE6AF6
:021DB000FCD75E
:0E1DB20012EE40F022EE40F0F86A019C5AEC6E
:0E1DC0000DF00CEC0FF05DEC0CF0FBD71200F8
:021DCE00FF0E06
:101DD000E350ACBA04D0AF6AAB8EAC8A949CACA290
:0A1DE000FED7AD6EF36EF46A120038
:061DEA00FF0EE350E84E7D
:101DF0001200000000D000D000D0E82EFAD7120068
:101E00003031323334353637383961626364656670
:011E100000D1
:041E11002533640011
:021E16001200B8
:021E18001200B6
:061E1A00EEEDEBE7DEDD5A
:101E2000DBD7BEBDBBB77E7D7B77303132333435F7
:101E3000363738394142434445467E0CB69ECCDAAB
:081E4000FA0EFECE3030300036
:00000001FF
